:020000040000fa
:080000000414040000000000dc
:020000040000fa
:1004000000000000000000000000000000000000ec
:1004100000000000000000000000000000000000dc
:1004200000000000000000000000000000000000cc
:1004300000000000000000000000000000000000bc
:10280000ffffff00ffffff000f532100807f240028
:1028100000018800000000000a0007001100070006
:10282000000020000000e000020032000000020072
:1028300000000000cc890200000000000040da0027
:102840000000fe004440a900403120000000e000ec
:102850000300320000002000a00188004440a800ce
:102860000000060080b52800010020001600370097
:1028700062004000e0804800910188009001ba00a9
:1028800062004000e0804800910188009002ba0098
:1028900062004000e08048000002eb006028e10098
:1028a00005003a008301e9000700330003800900b6
:1028b0000059eb00040037006128e10001003200fc
:1028c0000082eb0005000700910188001001ba00aa
:1028d0000200e000e6ff3a000000050091018800d8
:1028e0008002780062004000e08048003559ba005c
:1028f0008301e900080032002559ba008301e9008c
:10290000050032000400e000f4ff320015d9ba00df
:102910008301e900f1ff3a0000000600cc830400c7
:1029200000000000b483040000000000ac83040039
:10293000000000009e830400000000003a860400ae
:1029400000000000e6880400000000001888040071
:1029500000000000800078001104b1000300350081
:102960009101b10001003c000050a00000000600f1
:102970008001eb0002003700817178008301e800dc
:10298000828f5100fcff3a0000000600000378002f
:10299000800178000002eb000100370080597800c8
:1029a00084025100820f52000900320064c0780096
:1029b0000402e8000004e000f8ff3a008300780019
:1029c0008058eb0005804100808f5000fcff3a00ea
:1029d0000600780000000600800078001106b100b3
:1029e000030035009101b10001003c000050a1003e
:1029f0000000060080007800010037000000e800b9
:102a00001004e000fdff3a00010050000000060045
:102a1000800178000001780031407800005978008a
:102a20000004e000fcff3a0003007800000006000c
:102a3000040037000204e00001003a000000050035
:102a40000000e80010417800814f5100f9ff3a0082
:102a5000000006006022b800060220000000d0003e
:102a60008180d2000482d2008582d2000000a000c2
:102a70000202520083825a00030031000202420027
:102a800083824a000000a1000603e900f3ff3a0038
:102a900000000600881f7800000478005001be0086
:102aa0004000be0004004000858048000601490047
:102ab00087814900009cbe000294be000400e10032
:102ac0000588e1000690e1000798e100020031006e
:102ad000680044001008e8004f0478000000060079
:102ae000f4874700889fbe008a9fbe008c9fbe006f
:102af0008e1f78000205be000004be00d4b79f0000
:102b0000e5b79f00f6b79f0087bf9f000000eb006e
:102b1000c0b79f00b0b79f00a0b79f0090b79f00bd
:102b200080b79f000d042000bfb097004fb0970002
:102b3000000140000000e0000f003d004f08de00f3
:102b400000007100c0b79f009e00070001003d001b
:102b500012002000a100070001003d00120020002b
:102b6000a6000700b1000700b60007000f004000f4
:102b7000c8ff0700220037004f08de000006710082
:102b8000ccb79f008f00070001003d00120020001d
:102b90009200070001003d0012002000970007008e
:102ba000a20007000fb297009fb297002fb39700c3
:102bb000bfb39700a90007000000520081805a00af
:102bc00002015b0083815b0080b79f0091b79f008b
:102bd000a2b79f00b3b79f000007eb009f0007005c
:102be0000020e10001a8e10002b0e10003b8e1002b
:102bf000010031001e0020000e005600c0b79f00eb
:102c00004fb297000400e0000700350010002000dc
:102c1000010020006011b800080470008984700071
:102c20000a0571008b8571008d06e900beff3a0030
:102c30000400e00003003d00820007000f00400098
:102c400094ff07004fa897000000e00004003a003e
:102c50000fb497009fb497002fb59700bfb59700aa
:102c6000940007004f0778004f06be004f05be00d6
:102c70004f04be004f01b10000000600881f78001d
:102c800018002000881f780095ff07008f87e90053
:102c90004f04780000000600801feb0090ff070043
:102ca0008f87e90000000600889fbe008a9fbe0053
:102cb0008c1f78006e00070007003d0073000700be
:102cc000e00f5b00e08f5b0007003d003200070073
:102cd0000006eb00040037003400070002003d004e
:102ce0002a0007001c00200072000700e3ff070015
:102cf0000203be000002be000c00e0000100320032
:102d0000220007000400be000601be004f06780046
:102d10004f05be004f04be0000000600889fbe00a5
:102d20008a9fbe008c1f78005100070005003d00ff
:102d300056000700e00f5b00e08f5b0006003d00df
:102d4000040037001900070003003d006000b800d0
:102d50006011b8001000070056000700ceff070002
:102d60000203be000002be000c00e00001003200c1
:102d7000060007000400be000601be004f067800f2
:102d80004f05be004f04be00000006006000b80002
:102d90006011b8000000370004025000858258001e
:102da0000603590087835900000006000006eb0067
:102db000e00f5200e08f5a00e00f5b00e08f5b00f5
:102dc000000006000180400090b79f000001eb006a
:102dd0008fb097000100e0000000060002007000c4
:102de00090b79f000180400080b79f000001eb007a
:102df000ffa897000100e00000000600020070003c
:102e000080b79f00018040006faa9700cf20de00ae
:102e100001007000f0af9f0004024200250007008f
:102e20004f18de000002720000000600e4af9f00b1
:102e30000804440089844c000a054d008b854d0030
:102e4000000006003fb29700cfb297005fb3970033
:102e5000efb3970000fe2f00000006003fb0970080
:102e6000cfb097005fb19700efb197000000060068
:102e70000205be000004be00e00f5000e08f5800c5
:102e8000e00f5900e08f5900000006006000b80014
:102e90006011b80008045000898458000a055900e0
:102ea0008b8559001c002000e00f5200e08f5a0073
:102eb000000006000800be000a01be000000060077
:020000040000fa
:020000040005f5
:0457f800fe9300001c
:020000040000fa
:020000040005f5
:0457fc007f3e0000ec
:020000040000fa
:102ec00012010000100100000000000000080000d6
:102ed000d804000009000000010000000102000009
:102ee00000010000090200002000000001010000b4
:102ef00000c00000320900000400000000020000d1
:102f000008060000500000000705000081020000d4
:102f10004000000001070000050100000240000021
:102f20000001000004030000090400003403000055
:102f30004d00000069000000630000007200000006
:102f40006f000000630000006800000069000000de
:102f50007000000020000000540000006500000028
:102f600063000000680000006e0000006f000000b9
:102f70006c0000006f000000670000007900000096
:102f800020000000490000006e0000006300000007
:102f90002e0000003a0300004d0000006900000010
:102fa00063000000720000006f000000630000007a
:102fb00068000000690000007000000020000000b0
:102fc0004d0000006100000073000000730000006d
:102fd0002000000053000000740000006f0000009b
:102fe0007200000061000000670000006500000042
:102ff0002000000044000000720000006900000092
:1030000076000000650000007297000092970000b3
:1030100096970000ca97000000950000000000008d
:103020000000000001f900000000000000000000a6
:1030300009af000000000000010000000a1b0000b2
:1030400000000000010000000cc3000000000000b0
:10305000000000000daf00000200000000000000b2
:1030600010ff0000000000000000000011ff000041
:10307000000000000100000012ff0000000000003e
:103080000100000018ff0000000000000100000027
:1030900019ff0000000000000100000020ff0000f8
:1030a000000000000000000021ff00000000000000
:1030b0000000000022ff00000000000000000000ef
:1030c00023ff0000000000000000000024ff0000bb
:1030d000000000000000000025ff000000000000cc
:1030e0000000000026df00000100000000000000da
:1030f00031890000010000000000000029e5000007
:103100000000000000000000377300000000000015
:10311000000000003a25000003000000000000004d
:103120003b250000000000000000000000800000bf
:103130000402000020000000000000004d690000b3
:10314000637200006f630000687000004d61000052
:103150007373000020530000746f00007261000060
:1031600067650000202000002020000030300000b3
:1031700030310000256400000d0a000000770000d7
:10318000006c00006f6700002e6300007376000083
:103190000000000030310000323300003435000000
:1031a00036370000383900006162000063640000b7
:1031b00065660000002e00002e00000020200000a8
:1031c00020200000202000002020000020200000ff
:0431d00020000000db
:020000040000fa
:1031d4000400fa000000eb00000f7800060037003e
:1031e4009e007800a0f020008080400010c0b30052
:1031f400804878001e0fe800200020009e0f100079
:10320400f7ff34000040eb005ff0b7005a350700c9
:10321400e0fc2000280207000004e00034003a002b
:1032240011838000e0fc2000800878001183800076
:103234000000eb00d0009800118380000000eb0038
:10324400e0009800128380006000b80070019800cc
:1032540001099800128380006000b80010099800ea
:103264002109980011838000c0c5b300c05898009c
:1032740010002000000f7800070037001183800041
:103284001e00780000804000fc00400000c2b30033
:10329400804878001e0fe800a00020009e0f100058
:1032a400f6ff3400118380000000eb00c01098008a
:1032b4001183800000012000e01098001283800038
:1032c400c0788000d17880007011980001199800ae
:1032d40012838000c0788000d17880001019980093
:1032e40021199800100020001007980002003700f0
:1032f4000000eb00100798001e0090000080fa0008
:10330400000006001400fa00881f78006007980087
:103314007107980002579800135798006e009000a8
:103324004010900050079800a0002000100798005b
:103334006e00900080189000701090006e01900054
:1033440010199800211998007e00900060109000d8
:103354000080ea00300798005e0090000000e00062
:1033640009003a00ea00470012c0b3006e00900062
:103374009a0707000000e0000f003a00c001200097
:10338400100798000c0037005e0090006f0060008a
:103394000000e00008003200ea00470012c0b30059
:1033a4006e0090008d0707000000e00002003a0064
:1033b400c0012000100798001e009000fc0f500070
:1033c400bb0032001e0090000000e000b800320094
:1033d400ea0047006e009000700b07005047980009
:1033e4005e409000e24f5000b10032005e40900019
:1033f4000004e000a5003a006e009000e010900088
:1034040041079800ce009000f00320000080600087
:10341400400798001e5090000080fb00100f980099
:103424001e0890000000e000040032009e08900096
:10343400e18f500031003200990037004e009000b7
:10344400e80f5000960032004e0090000000d100ba
:103454000000a200610060000004e000900032005f
:103464000000eb0010079800d0c6b3001047980086
:103474000040eb00404798001c0037004e4090008d
:103484000080fb00ee0090007c0040000100400042
:1034940010407800104798004e4090000080fb00d8
:1034a400fe0090007c0040000100400010407800c5
:1034b400004f78001e4090000080fb0024fd0700b0
:1034c400000478001e80fb0021fd0700800f5400db
:1034d40003003200a000200010079800700037009d
:1034e4004e4090000040e800404798004e40900055
:1034f400ea4f5000e1ff3600690037004e009000ab
:10350400be009000010060000000e00064003a008a
:103514004e009000ef0f5000610032000000eb00fd
:1035240010079800d0c6b300104798007e009000a2
:10353400c0589000a0c2b30080cf500025003200d4
:103544000040eb00404798001f0037004e409000b9
:103554000080fb00ee0090007c0040000100400071
:1035640010407800104798004e4090000080fb0007
:10357400fe0090007c0040000100400010407800f4
:10358400004f7800a0c2b3009e4f1000110032001b
:103594001e4090000080fb00edfc07000004780052
:1035a4001e80fb00eafc0700800f54000300320079
:1035b400a000200010079800060037004e4090003d
:1035c4000040e800404798004e409000e74f50000c
:1035d400deff36007e009000c0609000a0c2b30001
:1035e40080cf50002e0032001e0090000000e0004a
:1035f4002b003a0080c0b300404798001f003700fa
:103604004e4090000080fb00ee0090007c004000e3
:103614000100400010407800104798004e40900090
:103624000080fb00fe0090007c0040000100400090
:1036340010407800004f7800a0c2b3009e4f1000e5
:10364400170032001e4090000080fb00c0fc070001
:10365400000478001e80fb00bdfc0700800f5400ae
:1036640003003200a0002000100798000c0037006f
:103674004e4090000040e800404798004e409000c3
:10368400ea4f5000deff3600050037000e50900070
:103694000004e00002003a000000eb00100798006c
:1036a4005e0090000000e8005007980045ff3700d6
:1036b4001e0090004f0478000080fa00000006000d
:1036c4001200fa005007980061079800624f9800b2
:1036d4000000eb00000f78005e009000900078007e
:1036e400410798004e009000505890000004e000fc
:1036f40003003a0060002000000f78007d003700ce
:103704005e00900080189000701090005e019000a0
:1037140010199800211998006e009000100078008c
:103724000000e00009003a0012c0b300ee0090006f
:103734005e009000a90607000000e00010003a00b7
:10374400c0012000000f78000d0037006e009000cb
:10375400100078006f0060000000e00008003200f4
:1037640012c0b300ee0090005e0090009b060700bc
:103774000000e00002003a00c0012000000f7800c1
:10378400ee0090005e009000840a070060479800f5
:103794006e4090000004e00003003200a00020000e
:1037a400000f7800530037005e0190006000b800fd
:1037b40070019800010998005e009000a00090003c
:1037c400100090005e0190003001980041019800c3
:1037d400de0090000000eb00d0009800de009000b6
:1037e4000000eb00e00098006e409000e14f5000b4
:1037f40003003a00a0002000000f780028003700e2
:103804005e00900030019000c00190004e009000d6
:103814003e10070010079800210798005ed0bf00f3
:103824000004e00006003200c51107000004e000b7
:10383400030032000080eb00000f98002f003700d7
:10384400de009000c1828800d2828000e382800082
:103854001e009000ae009000800f5100818f59002f
:103864000f0032000040eb005ff0b7004e00900004
:10387400100178001e009000ae009000fc34070098
:103884000004e00002003a0070002000000f7800fd
:103894001e009000ae009000d0828800e182880073
:1038a400de009000310890000010a100b0089800dc
:1038b400ee48900070c7b30080cf5000040032007f
:1038c400ee48900010c6b30080cf500005003a00c7
:1038d400de009000310890000000a000b0089800bd
:1038e40004003700de009000310890000000a100c1
:1038f400b00898009e007800010f98000e08900010
:103904000080fa00000006001c00fa00200f980056
:10391400320f9800430f98000040eb0020479800b6
:103924002e089000100f78001e0078004058900078
:103934000080fb00500f98005e089000e10f5000db
:10394400160032005e099000e30f510001003200be
:103954000900370080ff2f00f1ff200020079800a6
:1039640031079800f0ff2f00f1ff20004007980076
:10397400510798001100370080ff2f00010020003c
:103984002007980031079800f0ff2f000100200065
:1039940040079800510798000800370080ff200076
:1039a400010020002007980031079800f0ff2f0045
:1039b4000100200040079800510798002e0890004d
:1039c40030019000c00190006207980073079800ce
:1039d4006e019000fe0190001e0078001015070093
:1039e400000f9800110f98000e0990009e09900096
:1039f4004e009000de009000800f5100818f59002e
:103a040003003a0070c0b300204798001300370049
:103a14001e00780020099000b00990000e08900064
:103a24009e089000800f5100818f590002003e00d3
:103a340090c0b300204798000e0990009e099000a2
:103a44002e009000be009000800f5100818f59001d
:103a540002003900c0c3b300204798002e0890002c
:103a64000e0990009e0990003200980043009800cf
:103a74003e089000ce08900061005000e08058009d
:103a8400300f9800410f98003e089000ce08900037
:103a9400e00f5000e08f5800030032002e409000e9
:103aa4000004e000c5ff32002e4090000080fb00bf
:103ab4000080fa00000006000400fa0010079800d5
:103ac4000040eb00004f78009e0090000040eb00a7
:103ad400d05898009e00900080a6200080087800ae
:103ae4002c330700e14f50000300320050c0b300f4
:103af400004f78000d0037001e0090000e000700f4
:103b0400004f78001e04e00008003a001e009000f8
:103b140096000700004f78001e04e00003003a00fe
:103b24009e00900010c0b300d05898001e80fb0087
:103b34000080fa00000006000c00fa00300798002c
:103b44000040eb00304798003e00900010017800e0
:103b54006000b80046340700e14f50000300320013
:103b640070c0b300304798007c0037003e009000de
:103b740010007800000f78001e007800e0f8930031
:103b840050c5b30080cf500034003a001e007800c6
:103b9400f0f89300a0cab30080cf50002f003a0081
:103ba4003e0090001000780061032000c229070045
:103bb4008040780060c4b30080cf500027003a00f2
:103bc4003e0090001000780071032000ba2907001d
:103bd4008040780010c4b30080cf50001f003a002a
:103be4003e0090001000780081032000b2290700f5
:103bf4008040780040c5b30080cf500017003a00e1
:103c04003e0090001000780091032000aa290700cc
:103c14008040780010c3b30080cf50000f003a00fa
:103c24003e0090001000780061022000a2290700e5
:103c34008040780090c2b30080cf500007003a0063
:103c44003e0190006000b800100198002101980026
:103c5400be00900020c0b300c05898003e00900001
:103c640010007800200798002e009000e0f89300e0
:103c740050c5b30080cf500005003a002e009000dc
:103c8400f0f89300a0cab30080cf500003003200c4
:103c940040c0b30030479800300037002e00900039
:103ca400c0a0910030a091003e0190001001980046
:103cb400210198002e009000a0c093002147980095
:103cc4002e4090000080fb00400798004e009000ba
:103cd400ee0f50001f003e0010002000ce009000a8
:103ce4000100dd005007980000052400de0090006c
:103cf400008060000000e0000e003a000080210017
:103d0400de009000008060000000e0000d003a003a
:103d1400de009000628060000000e00001003a00d4
:103d24000c003700be00900010c0b300c0589800cb
:103d34000a003700be00900020c0b300c0589800ad
:103d440006003700be00900030c0b300c058980091
:103d54000200370040c0b300304798003e40900056
:103d64000080fb000080fa00000006001800fa0042
:103d7400200f98000040eb00604798002e08900048
:103d8400100178002e089000a00090001000900010
:103d9400b7330700e14f50000300320070c0b30096
:103da40060479800ed0037002e089000100078005e
:103db400200798002e009000e0f8930050c5b3004f
:103dc40080cf500005003a002e009000f0f89300d8
:103dd400a0cab30080cf50000300320030c0b3004b
:103de40060479800dd0037002e089000100078002e
:103df400e100200039290700000f78002e08900008
:103e040010007800d10020002b29070080407800a2
:103e14002e089000315898002e0890001001900050
:103e2400a00190001e007800010020000200400064
:103e3400838048002e0990003001980041019800c9
:103e44002e08900010007800010120001a290700b4
:103e5400804078002e089000215898002e08900089
:103e640010007800610120001c2907008000780000
:103e74002e089000410898002e08900040089000f9
:103e84000000e00007003a002e08900010007800bf
:103e9400410220002b290700800078002e089000a2
:103ea400410898002e08900030019000c001900055
:103eb4002e089000205890008080fb002e0890006f
:103ec400400890000088b900010020000200400072
:103ed400838048002e0990005001980061019800e9
:103ee4002e0890001000780011012000fb28070024
:103ef400800078002e089000110898002e08900089
:103f04001000780031012000f4280700010020008f
:103f140060079800710798006e009000fe00900002
:103f2400e00f5000e08f580006003a002e08900081
:103f340010007800010220000229070060079800a1
:103f4400710798002e08900010007800b10020003e
:103f5400e2280700100798001e0090000000e0000f
:103f6400040032001e009000610060000004e000c4
:103f74000300320030002000300f98007a00370030
:103f84002e08900010089000c500dd001e0090006f
:103f9400008040000000e9001e01900011000900ab
:103fa4000280d80001002000000f9800110f980033
:103fb4002e089000205890008080fb002e0890006e
:103fc400400890000088b9001e0040006101b8005c
:103fd4000e0890009e089000020140008381480072
:103fe4006e009000fe009000020050008380580094
:103ff40040079800510798002e0890003058900010
:104004000081fb00030020004e009000de009000c1
:104014008ffa07002e0990002009980031099800b2
:104024002e08900020099000b009900040ff200065
:1040340001002000800f5100818f590004003e00d0
:10404400ae08900010c0b300c05898000f003700ad
:104054002e08900020099000b009900040ff2f0026
:1040640001002000800f5100818f590004003e00a0
:10407400ae08900020c0b300c05898000300370079
:10408400ae08900030c0b300c05898002e089000cd
:1040940040589000e34f50001b003a002e08900057
:1040a40010007800c1022000a6280700c07888000c
:1040b400d17888002e0890001000780001032000b9
:1040c400a0280700007988002e08900010007800ce
:1040d4002103200081280700f07888002e08900032
:1040e40050019000e00190000e0890009e0890009e
:1040f40002004000838048002e099000700198005f
:10410400010998000f0037006000b800c0788800eb
:10411400d17888002e08900050019000e0019000b2
:104124002e089000100890004400de0001002000da
:1041340002004000838048002e099000700198001e
:10414400010998009e00900000202000808f5000fc
:104154000200320030c0b300604798006e40900007
:104164000080fb00300f98003e0890000080fa00a9
:10417400000006005400fa00207f9800621f980097
:10418400731f9800012798007c004700500798008f
:10419400de00900080a620008008780076310700b9
:1041a4007c310700e14f5000030032000080eb0037
:1041b400302798002d03370082a620006000b80045
:1041c400ab3207000004e00003003a008080eb00fb
:1041d40031279800250337005e0090001000780016
:1041e400600798006e009000e0f8930050c5b3009b
:1041f40080cf50004d003a006e009000f0f893001c
:10420400a0cab30080cf500048003a005e0090007e
:104214001000780061032000272807008040780000
:1042240060c4b30080cf500038003a005e009000b4
:1042340010007800710320001f28070080407800d8
:1042440010c4b30080cf500030003a005e009000ec
:1042540010007800810320001728070080407800b0
:1042640040c5b30080cf500028003a005e009000a3
:1042740010007800910320000f2807008040780088
:1042840010c3b30080cf500020003a005e009000bd
:1042940010007800610220000728070080407800a1
:1042a40090c2b30080cf500018003a002e789000de
:1042b4000000fb00202798002e2190000200e0005f
:1042c40007003200ae219000e18f5100010032005e
:1042d400160037000082eb0034279800e302370011
:1042e4005e0090006011b80012009800230098004e
:1042f4005e0090009dfe07000004e0000b00320009
:104304000080eb0030279800d802370080a62000f8
:10431400500f98005e089000c0a0910030a091005a
:104324005e01900010019800210198002e78900001
:104334000000fb00102798009e2090000100e00080
:10434400e90132001e219000e10f5100010032000a
:10435400ec0137005e08900050a19100e0a19100ab
:10436400320f9800430f98003e099000ce09900048
:104374008003210001002000800f5100818f59002b
:1043840024003e00de00900010c0b300c058980026
:10439400de08900010c0b300a0c09b0013c0b3009f
:1043a40082a620006000b800203307000004e0006b
:1043b40003003a008081eb0033279800ab023700fa
:1043c4003e099000ce0990007002210001002000f7
:1043d400800f5100818f590004003600de009000e8
:1043e40020c0b300b058980003003700de009000ee
:1043f40010c0b300b058980080a62000022020000e
:104404008000eb0059f9070020c3b300a2eab7000b
:10441400480037003e099000ce099000f0d52f00e7
:10442400f1032000800f5100818f59003e003e00af
:10443400de00900020c0b300c0589800de08900051
:1044440060c0b300a0c09b0013c0b30082a62000cc
:104454006000b800f53207000004e00003003a00f1
:104464000082eb0034279800800237003e09900058
:10447400ce09900080de2f00f1ff2f0002004000e3
:1044840083804800100f9800210f9800de009000f0
:1044940010c0b300b05898000d0037005e009000c3
:1044a400305890000080fb000000400080407800fd
:1044b4005e009000315898001e089000ae089000ed
:1044c4008100d1000080d300100f9800210f9800c4
:1044d4001e099000ae099000d0fe2f0001002000bc
:1044e400800f5100818f5900ecff3e005e00900068
:1044f400b058900000c8b30080cf500003003600cd
:104504000080eb00302798005802370080a6200076
:10451400022020008000eb0014f9070060c3b30000
:10452400a2eab700030037008080eb00312798002f
:104534004e0237005e009000305890000080fb006f
:10454400000040006101b9003e089000ce089000d0
:104554000201400083814800f0fd2f00f1ff2f008d
:10456400020040008380480020079800310798002b
:104574005e00900040589000e14f500009003a005e
:104584005e009000305890008080fb0050152000a1
:104594000088b9000080e800cf80de00008fbe00f4
:1045a400070037005e009000305890000080fb0048
:1045b4004800dd000080e800cf80de00008fbe00f0
:1045c4002e009000be0090003e014000ae814800e5
:1045d4000200be0061005000e08058001e01be00d1
:1045e4001bf907002007980031079800b0ceb300ec
:1045f40068eab700c0c3b30069eab70000c9b300f2
:104604006aeab700d0c4b3006beab70030c4b300a1
:104614006ceab70080c4b3006deab70000c5b3000c
:104624006eeab70000c2b3006feab70060c4b3001b
:1046340070eab70010c4b30071eab70040c5b30014
:1046440072eab7000040eb0073eab70020c0b30081
:1046540074eab7005e0090003058900075eab70025
:1046640080c0b30076eab7000040eb0077eab700f9
:104674005e009000a00090001000900068004000d0
:10468400e08048005e0190003001980041019800ec
:1046940020c0b30078eab700de00900020c0b30069
:1046a400a05898000040eb0079eab70020c0b3009e
:1046b4007aeab700de0090000020200090089800fd
:1046c4000040eb007beab7000040eb007ceab70057
:1046d40080cfb3007deab7002e0090007eeab700d9
:1046e4002e009000be009000c809dd004800de00e6
:1046f40000807100c808de007feab700ae009000b9
:104704005e00900041089800f0c3b30080eab7004f
:104714000040eb0081eab70000c0eb0082eab7007a
:104724000040eb0083eab7005e009000a000900018
:104734001000900084eab7005e009000a000900092
:1047440010009000480add004800de0000007200fe
:10475400c808de0085eab7005e009000a000900063
:10476400100090004008de000100200086eab70037
:104774005e009000a0009000100090004808de0049
:104784000100200087eab7003e08900088eab700dd
:104794003e089000ce0890004809dd004800de0085
:1047a40000007100c808de0089eab7003e089000e6
:1047b400ce0890004008de00010020008aeab7001d
:1047c4003e089000ce0890004808de00010020005a
:1047d4008beab7000040eb008ceab7000040eb0026
:1047e4008deab70090c2b3008eeab7006e1890004d
:1047f4008040780000c0eb0000c060008feab70082
:104804006e189000fe1890004027980051279800d9
:104814004e209000de209000e00f5000e08f580002
:1048240006003d004e219000de219000f20fb00002
:104834000380b00042279800532798004e2190002f
:10484400de219000481add004810de0000007200ee
:10485400c898de008040780000c0eb0000c0600013
:1048640090eab7006e189000fe1890006027980038
:10487400712798006e209000fe209000e00f5000f9
:10488400e08f580008003d00f0ff2f0001002000d9
:104894006e219000fe2190000201400083814800b7
:1048a40062279800732798006e219000fe219000e3
:1048b4004098de00cf80de008040780000c0eb002e
:1048c40000c0600091eab7006e189000fe189000d6
:1048d400002f9800112f98000e2890009e28900019
:1048e400e00f5000e08f580008003d00f0ff2f005b
:1048f400f10f20000e2990009e2990000201400033
:1049040083814800022f9800132f98000e299000ed
:104914009e2990004898de00cf80de008040780019
:1049240000c0eb0000c0600092eab7000e209000c7
:104934000000e0002f0032000040eb0026efb7003b
:104944001100370026cfbf000080fb00b202200018
:104954000001410026cfbf000080fb0080007800ea
:104964000e209000008040001040780080407800c5
:1049740080a62000000041000148780026cfbf0037
:104984000040e80026efb70026cfbf000080fb0000
:10499400800078000e2090000080400010407800d5
:1049a4000004e0000f00320026cfbf00ea4f5000a1
:1049b400e4ff36000b00370062f220001241780059
:1049c4000280fb00b10220008080400080a620000d
:1049d4008080400000c2b300804878000240e800b4
:1049e40026efb70026cfbf00ea4f5000f2ff360093
:1049f400110037000040eb0026efb7000b00370032
:104a040026cfbf000080fb00b10220008080400060
:104a140080a62000808040000040eb0080487800a1
:104a240026cfbf000040e80026efb70026cfbf0026
:104a3400ea4f5000f2ff360060c4b3009eeab700ac
:104a440010c4b3009feab70040c5b300a0eab700a2
:104a540010c3b300a1eab70000c2b300a3eab700d1
:104a640000c2b300a4eab70000c2b300a5eab700cd
:104a740050c5b30066ecb700a0cab30067ecb7003a
:104a84005e00900030019000c00190005e00900034
:104a9400205890008080fb005e0090004008900049
:104aa4000088b90001002000020040008380480013
:104ab4005e01900050019800610198005e00900032
:104ac400a0009000100090008041eb0082a620001e
:104ad400563107000004e0000d003a008081eb002d
:104ae40033279800e10037005e0090009ffc070028
:104af4000004e000060032000082eb003427980036
:104b0400da0037000080eb0030279800d700370028
:104b140080a62000022020008000eb0093f707000d
:104b240080cfb30068eab70000c0eb0069eab700c1
:104b340000c0eb006aeab7005e00900040589000a5
:104b4400e24f500002003a0000c0eb006beab700ed
:104b54005e009000205890000080fb000000e900f7
:104b640040079800150037005e0090003001900067
:104b7400c00190005e009000c00890004e009000bc
:104b84000088b90001002000020040008380480032
:104b94008041eb0082a62000243107000004e000dd
:104ba40003003a008080eb0031279800af00370003
:104bb4004e0090000000e900400798004e0090006d
:104bc400e10f4000e8ff3a006000b800405388005d
:104bd400515388005e009000c000900030009000a7
:104be4000040e80026efb7001f0037005e00900089
:104bf400205890000080fb000000e9004007980066
:104c04001300370026cfbf000081fb005e00900038
:104c1400c00890004e0090000088b90000004100d8
:104c2400010020008041eb0082a62000ff30070035
:104c34000004e00003003a000081eb0032279800f2
:104c44008a0037004e0090000000e90040079800f9
:104c54004e009000e10f4000eaff3a0026cfbf006b
:104c64000040e80026efb70026cfbf000082fb001b
:104c7400050020005e00900030019000c00190000b
:104c84005e009000400890000100200002004000f7
:104c940083804800800f5200818f5a00d3ff39006f
:104ca4005e009000100890004500dd00f01fb00089
:104cb4004900de000100200070079800010f9800f1
:104cc40010c0b30026efb700130037005e00900059
:104cd40050019000e001900026cfbf000080fb004f
:104ce4000100200002004000838048008041eb0066
:104cf40082a62000cd3007000004e00003003a0043
:104d04008081eb00332798005800370026cfbf007e
:104d14000040e80026efb70026cfbf000081fb006b
:104d2400030020007e0090008e089000800f510048
:104d3400818f5900e5ff39000e2090000000e0004b
:104d44003d0032000040eb0026efb7000f003700b3
:104d540026cfbf000081fb0026cfbf000080fb00f0
:104d6400800078000e209000008040001040780001
:104d74008040780080a620000000410001487800af
:104d840026cfbf000040e80026efb70026cfbf00c3
:104d94000080fb00800078000e209000008040001e
:104da400104078000004e0000d00320026cfbf0060
:104db400ea4f5000e6ff36000900370062f2200097
:104dc400124178008280fb0080a620008080400091
:104dd40000c2b300804878000240e80026efb70024
:104de40026cfbf00ea4f5000f4ff360080c0b30066
:104df40073eab70010c1b30079eab70010c1b30079
:104e04007beab70010c1b3007feab7005e009000f0
:104e1400e0009000500090008041eb0082a620004a
:104e2400823007000004e0000e003a000082eb002c
:104e3400342798000d0037005e009000e0009000d9
:104e4400500090008041eb0082a6200077300700dc
:104e54000004e00003003a000080eb0030279800d3
:104e6400020037008000eb00312798003e209000bc
:104e74000080fa00000006001200fa0060079800a3
:104e8400710798006e009000900078005107980018
:104e94006e00900010199000a0199000028fbe00bf
:104ea4007e009000100078004400de00004f98005f
:104eb4005e009000405890000080fb00000f9800b6
:104ec4008e099000e18f51001f0035000e089000fc
:104ed400e20f50000e0034008e089000e38f500063
:104ee40001003200180037005e009000b0589000b6
:104ef4000e4890000080fb000181fb0011000900b6
:104f04000280d8008000fd00004f98000e0037009a
:104f1400c0788000d1788000be0f1000ae8f1800da
:104f2400090032005e009000b05890000e489000d6
:104f34000080fb000181fb00110009000280d80001
:104f44008000fd00004f98001e01be005e0090002e
:104f54006e0a070020079800310798005e00900051
:104f6400100278000e4890000081fb00030020002e
:104f74002e009000be009000020040008380480094
:104f84008041eb0004017800283007000004e000b1
:104f940003003a000040eb00104f98000200370075
:104fa40010c0b300104f98001e4890000080fb0012
:104fb4000080fa00000006001800fa00700798004c
:104fc400010f9800120f98000000eb00000f78000a
:104fd4001e089000405890000080fb00300f98009d
:104fe4003e089000e20f500010003200be0890000e
:104ff400e38f5000040032003e089000e10f50009f
:10500400130032001a003700f0ff2f00f1ff2000d8
:10501400100798002107980080ff2f00f1ff20005f
:10502400300798004107980011003700f0ff2f0067
:1050340001002000100798002107980080ff2f002e
:10504400010020003007980041079800080037004d
:10505400f0ff2f000100200010079800210798009e
:1050640080ff2000010020003007980041079800cd
:105074007e0090008e089000e00f5000e08f5800f2
:10508400070032007e0190008e099000100020007d
:1050940001002000800f5100818f59003d003a002b
:1050a40020002000000f78003c0037007e019000b3
:1050b4008e0990001e089000590f070050079800b1
:1050c400610798005e019000ee0190001e009000c0
:1050d400ae009000800f5100818f590003003a0008
:1050e40010002000000f78002a0037005e009000b6
:1050f400ee009000e00f5000e08f580007003200ef
:105104005e019000ee0190001000200001002000dc
:10511400800f5100818f590003003a0020002000c5
:10512400000f78001b0037005e019000ee01900034
:105134003e009000ce009000800f5100818f5900f6
:105144000200390020002000000f78008040eb00ae
:105154006022b8007e0190008e0990001e08900025
:10516400031107000001be001e009000ae00900075
:10517400800f5100818f590002003a001000200076
:10518400000f78005e009000ee0090007007980019
:10519400010f98001e00e000c4ff320011c0b300ec
:1051a4006022b8006011b8001e089000f0100700db
:1051b400210020009e8f100003003a001000200000
:1051c400200f9800020037008000eb00210f9800a8
:1051d4002e0890000080fa00000006002000fa006b
:1051e400300f9800410f9800225f98003e0890000d
:1051f40090007800110f98003e0890007011900004
:105204008019900052079800630798003e089000a8
:1052140010199000a0199000120798002307980015
:105224004e089000100078004400de0010479800fb
:105234001e089000405890000080fb00700f9800fa
:10524400fe099000e18f5100270035007e08900090
:10525400e20f500012003400fe089000e38f50006b
:1052640001003200200037001e089000b058900062
:105274001e4090000080fb000181fb00110009002a
:105284000280d8008000fd001047980080ff2f00a6
:10529400f1ff200030079800410798001200370002
:1052a4005e009000ee009000e00f5000e08f580088
:1052b400090032001e089000b05890001e40900073
:1052c4000080fb000181fb00110009000280d8006e
:1052d4008000fd001047980080ff2f00010020008f
:1052e40030079800410798002e5890000004e00011
:1052f40005003a004e089000100078006f0060002e
:105304000000e0008c003a001e4090000004e00021
:1053140004003a004e08900010007800ef0f50008f
:1053240003003e002e5890000004e00020003200ec
:105334002e5890000004e0000a0032004e0890004d
:10534400900078001e089000305890000080fb0008
:105354004401dd00110009008280d800004f78006c
:105364001100370010c0b300004f78000e00370062
:105374001e019000ae0190001e089000a80e0700c8
:1053840010079800210798001e019000ae019000bc
:105394003e009000ce009000800f5100818f590094
:1053a400030031001e4fe9001e04e000f0ff3a0044
:1053b4001e019000ae0190003e009000ce009000cf
:1053c400800f5100818f5900580031003e08900031
:1053d4001e019000ae019000121898002318980046
:1053e4001e019000ae0190001e08900047090700be
:1053f40070079800010f9800c2788000d37880006d
:105404001e009000ae009000820f5000838f580061
:1054140014003a001e4090000081fb0003002000ad
:105424007e0090008e0890000201400083814800b5
:105434001e0890008008900070009000800f5100ba
:10544400818f5900070039001e08900040589000d1
:10545400e34f5000030032000000eb00200f9800df
:105464003e0037005ed0bf000004e00006003200ba
:10547400b30a07000004e000030032008001eb00df
:10548400630f9800370037000000eb00c0828800eb
:105494000040eb005ff0b7001e0890001002780097
:1054a4001e4090000081fb00030020007e0090005d
:1054b4008e089000020040008380480004017800b8
:1054c400eb2d0700e14f5000030032000000eb0019
:1054d400200f9800100037002e5890000004e000c0
:1054e4000a0032001e089000100078008000780046
:1054f4004e089000100078006f0060004500dd0049
:1055040000804000200f9800030037001e08900020
:1055140010007800200f98000080eb008080eb00e2
:10552400d0828800e18288000c0037000000eb0084
:10553400200f9800090037001e0890001000780022
:10554400800078004e089000100078006f00600022
:105554004500dd0000804000200f98002e089000d8
:10556400600f98006e0890000080fa0000000600aa
:105574001400fa0070079800010f98002257980051
:105584000000eb00000f78000040eb00204798007b
:105594000d0037002e4090000081fb002e4090004b
:1055a4000080fb00fe0090007c00400001004000f1
:1055b4009040780063004700017178002e4090000d
:1055c4000040e800204798002e409000ea4f500029
:1055d400f0ff36001e00e00017003a000e089000ad
:1055e4008000eb00010878008e0890007e00900097
:1055f4005a0007000004e0000d003200e3004700f9
:10560400ae5190000e0990007e009000c500070086
:105614000080fb00000f78001e00e00006003a0046
:105624007e00900007000700000f7800020037009a
:1056340010012000000f78001e0078000080fa009e
:10564400000006001400fa00700798007e00900025
:105654004010900060079800e80047007e0090002a
:1056640010080700300798003e0090000000e0009a
:1056740037003a00ec0047007e0090006303070007
:10568400000f78004e009000de009000800078004b
:105694001e007800510898004e009000de00900033
:1056a40002002000f3ff200000027800810278004d
:1056b400020078008300780000016200018062002b
:1056c4006102b800040f9800150f98000e089000ae
:1056d4009e089000c000dd0000002000000f98002c
:1056e400110f98000e0890009e0890006112b800f7
:1056f400040f9800150f98000e0990009e09900061
:105704000200700083807000100798002107980041
:105714001e009000ae0090004008de000100200052
:1057240010079800210798009e0090001e00780042
:1057340021089800ec0047007e009000cefd070091
:10574400e14f500002003200800020003007980032
:105754003e0090000080fa00000006001200fa00eb
:10576400600798007107980010c0b300204f98009c
:105774006e00900080189000701090006e019000f0
:10578400101998002119980012c0b300fe0090006f
:105794006e00900091fe0700000f78001e00e000ec
:1057a4004f003a00c0c1b300204f980052003700a8
:1057b4000040eb00104f98007e00900090007800ad
:1057c400310798000041eb00fe0090006e0090004d
:1057d40082fe0700000f78001e0078001040780059
:1057e400004f98007e009000100078008000e800d0
:1057f4007e009000010878000e489000fb4f4000a6
:10580400030032000e4890000004e00008003a0053
:105814001e00e000060032001e4890000040e80030
:10582400104f98001e4890000004e000e5ff32008d
:105834001e00e00022003a006e0090001019900053
:10584400a01990001207980023079800c2788000de
:10585400d37880001e009000ae009000820f5000ac
:10586400838f580003003a0020c0b300204f9800f3
:105874001b0037006e0090001e019000ae019000e6
:10588400320098004300980011c0b3006e009000ed
:1058940095000700f24f500003003a0020c0b30007
:1058a400204f98000e0037007e009000be0190004b
:1058b400030878000040eb00204f980008003700f0
:1058c4001e489000e14f500005003a000040eb00f4
:1058d400204f98007e009000be00900001087800e0
:1058e4002e489000e14f5000b1ff32007e0090003e
:1058f4003e019000020878002e4890000004e00069
:1059040003003a0013002000030f98000200370040
:105914000000eb00000f98000e0890000080fa00d1
:10592400000006000e00fa002007980031079800d6
:1059340042079800234f98000040eb00204798004e
:105944002e00900080189000701090002e0190009e
:10595400101998002119980012c0b300ce009000cd
:105964002e0090001dfe0700000f78001e00e000ce
:1059740003003a00c0012000600798005700370078
:105984001e007800b2002000be009000fef3070065
:105994002e489000f24f500004003a009e00780018
:1059a40000c1b300b0489800030037009e0078009f
:1059b40000c2b300b04898009e0078000040eb009d
:1059c400c04898009e0078000000eb00a0089800f2
:1059d4009e0078000000eb00d00898001e017800bb
:1059e4006000b80060099800710998009e00780072
:1059f40020cbb300d04898009e0078008027270071
:105a0400f00098009e007800002b23008008980086
:105a14002e489000f24f50000a0032009e00780099
:105a2400002b2300900898009e0078009027270000
:105a3400b00898009e007800002b2300c00898004e
:105a4400090037009e0078000000eb0090089800e1
:105a54009e0078000000eb00b00898009e007800db
:105a64000000eb00c00898001e007800f0089000c9
:105a7400600890002e0190001009980021099800f8
:105a84001e007800f00090002e009000410898005d
:105a94001e007800800890002e00900051089800a5
:105aa4001e007800304890008080fb002e0090009b
:105ab400611098004e009000900078002e00900035
:105ac40041109800ce0090002e009000eafc0700e0
:105ad4002e4090000080fb00600798006e0090004c
:105ae4000080fa00000006001000fa005007980039
:105af400414f98005e0090009000780041079800a4
:105b04005e00900030019000c001900022079800d0
:105b1400330798005e0090004700070020079800b4
:105b2400310798002e009000be009000e00f500056
:105b3400e08f580003003a00230120007307980007
:105b44003a0037004e00900040589000e14f50005a
:105b540008003a008040eb0084ff2000050020008c
:105b64002e019000be0190004e009000800e0700b0
:105b7400130037004e00900040589000e24f500050
:105b840008003a008040eb0084ff2f00050020004d
:105b94002e019000be0190004e009000740e07008c
:105ba400070037008040eb0084ff2f00f5ff200042
:105bb4002e019000be0190004e0090006c0e070074
:105bc4005e00900030019000c0019000028fbe0082
:105bd4008040eb002e029000be0290001e01be0029
:105be4004e009000620e07005e0090002e019000af
:105bf400be01900032009800430098004e48900087
:105c0400e14f500007003a002e019000be019000c1
:105c14004e009000f90607000080fb007007980012
:105c2400020037008001eb00730798007e009000ab
:105c34000080fa00000006001a00fa00300f9800f5
:105c44006000b800000f9800110f98003e08900003
:105c540090007800210f98003e08900030019000d9
:105c6400c001900062079800730798002e08900006
:105c7400405890000080fb00400f9800ce0990002f
:105c8400e18f5100160035004e089000e20f5000dd
:105c94000c003400ce089000e38f50000100320065
:105ca4000f003700e0ff2f00f1ff200020079800cd
:105cb40031079800f0ff2f00f1ff2000008fbe0095
:105cc40007003700e0ff2f000100200020079800a4
:105cd40031079800f0ff2f0001002000008fbe0064
:105ce4006e019000fe0190001000200001002000d1
:105cf400800f5100818f590004003e0020002000d5
:105d04000100200060079800710798006e01900060
:105d1400fe01900042079800530798006e0190001e
:105d2400fe0190002e0890003d0c0700380037005b
:105d34006e019000fe0190002e089000380c0700c0
:105d4400000f9800110f98000e0890009e08900014
:105d5400be0f5000ae8f580004003a006000b80037
:105d640060079800710798002e0037000e08900015
:105d74009e089000e00f5000e08f58002900320088
:105d84006e009000fe00900061004000e08048003a
:105d940060079800710798000e0990009e09900012
:105da4002e009000be009000800f5100818f59009a
:105db400080032002e08900020099000b0099000dd
:105dc4006e009000fe009000800f5100818f5900fa
:105dd40004003e002000200001002000600798001d
:105de400710798006e019000fe0190004e00900033
:105df400de009000800f5100818f590004003a00aa
:105e04006000b8006007980071079800050037002b
:105e14006e009000fe009000e00f5000e08f5800ec
:105e2400c3ff3a006e009000fe0090000080fa006c
:105e3400000006000c00fa004007980080042000cf
:105e4400100798004e009000401090003007980012
:105e54004e00900030089000610060000000e000f7
:105e6400310032005ed0bf000004e00006003200c2
:105e7400330807000004e000030032000080eb0058
:105e840050079800480037004e009000100078003a
:105e940011c0b3006022b8006011b800b40d07004f
:105ea400e60047004e00900058010700000f7800fc
:105eb4001e00e00005003a000080eb001007980087
:105ec4001e00900050079800370037001e0078002d
:105ed40038000700000000004e009000a008900069
:105ee400100890001e01780060099800710998005c
:105ef400e60047004e009000dffb07000004e000ce
:105f0400030032000000eb00100798000200370085
:105f14000080eb0010079800ce009000310890003c
:105f24000000a100b00898000000eb0020079800d2
:105f340012003700ae009000600320000088b90012
:105f44008000780080e62000808040004e009000b1
:105f5400808f500006003a00ae009000a0f02000b0
:105f64008080400010c0b3008048780006003700ed
:105f74002e0090000000e800200798002e009000fa
:105f8400e20f5000ebff36009e00900080042000da
:105f9400808f500002003a000000eb0010079800c8
:105fa4001e009000500798005e0090000080fa00e8
:105fb400000006000800fa00300798003e00900038
:105fc400300890007f406000504798003e009000e9
:105fd400b0089000007e2000008060004500de00d4
:105fe400404798003e009000b008900000802f00c9
:105ff400008060004b00de00304798003e009000b7
:10600400400890007f406000204798003e009000c8
:10601400c0089000001e2000008060004500de00e3
:10602400104798003e009000c008900000e02f0048
:10603400008060004900de00004f78005e40900060
:10604400fc4f500004003e005e4090000040e80019
:1060540050479800280037000040eb005047980054
:10606400ce409000a0c3b30080cf500004003e0097
:106074004e4090000040e800404798001e00370062
:106084000040eb00404798003e409000f64f50001f
:1060940004003e003e4090000040e8003047980075
:1060a400150037000040eb00304798002e40900068
:1060b400fd4f500004003e002e4090000040e800d8
:1060c400204798000c00370010c0b3002047980008
:1060d4001e409000eb4f500004003e001e40900014
:1060e4000040e800104798000300370010c0b300d8
:1060f400104798001e4fe8005e4090008080fb002f
:106104003e009000310898003e009000b0089000d6
:106114004e4090000080fb004500dd008080700050
:106124003e009000310898003e009000b0089000b6
:106134003e4090000080fb004b00dd00808070003a
:106144003e009000310898002e4090008080fb00b3
:106154003e009000410898003e009000c008900066
:106164001e4090000080fb004500dd008080700030
:106174003e009000410898003e009000c008900046
:106184001e80fb004900dd00808070003e0090000e
:10619400410898000080fa00000006000c00fa0094
:1061a40040079800510798000040eb00004f78002a
:1061b4005e009000100078006f0060000000e000b6
:1061c40010003a005e009000100078000000e0002b
:1061d4000c0032004e009000801890007010900067
:1061e4004e019000101998002119980012c0b300b4
:1061f400de0090004e009000f8fb07003007980086
:10620400050037000041eb00de0090004e009000d6
:10621400f2fb0700300798003e0090001040780021
:10622400304798003e0090000000e0000300320078
:106234003e4090000004e00003003a0020c0b30098
:10624400104798006d0037003e409000fb4f40001f
:1062540003003a0010c0b3001047980067003700ed
:106264003e009000b0489000314798000040eb0099
:1062740040479800140037004e4090008080fb0097
:106284003e009000008040001040780020479800b5
:106294002e4090000080fb00cef1070020479800bc
:1062a4009e80fb002e4190004e00900001004000b3
:1062b4007c004000024878001e4fe8004e409000e9
:1062c4000040e800404798004e409000e74f5000df
:1062d400e9ff36003e009000b04890003147980036
:1062e4003e00900000489000204798000040eb00da
:1062f40040479800150037004e4090000080fb0096
:10630400be0090006800400001004000104078008a
:10631400204798002e4090000080fb00adf107005c
:10632400204798009e80fb002e4190004e00900074
:10633400010040007c004000024878001e4fe80045
:106344004e4090000040e800404798004e409000c6
:10635400e24f5000e8ff36005e00900090007800a5
:106364004e009000411098003e00900010407800cc
:10637400304798003e409000fb4f400003003a0035
:1063840010c0b30010479800020037000040eb0033
:10639400104798003e009000f008900060089000bc
:1063a4004e01900010099800210998003e009000c9
:1063b400ad1f07004e0190001001980021019800c4
:1063c4003e009000b00890004e00900041089800f4
:1063d4003e009000c00890004e00900051089800c4
:1063e4003e009000b0489000314798003e40900035
:1063f4008080fb004e009000611098001e409000c9
:106404000080fb000080fa00000006000a00fa0089
:1064140020079800310798002e0090008018900003
:10642400701090002e019000101998002119980006
:1064340012c0b300be0090002e00900067fb07005e
:10644400100798001e0090000000e00003003a00ce
:106454000000eb00400798002c0037001e0090005d
:1064640010407800004f78001e04e00002003a005b
:106474000000eb00100798001e0090000000e000f0
:106484002000320051ceb3009ecf100003003a002a
:106494000000eb00100798001a0037001e0090005f
:1064a400b0489000014f7800130037003e00900080
:1064b400100078008000e8003e0090000108780099
:1064c4000041eb00be0090002e00900043fb07004b
:1064d400100798001e0090000000e00003003a003e
:1064e4000000eb0040079800080037001e009000f1
:1064f400b0489000014f7800f0c0b3009e4f1000e8
:10650400eaff32009e009000410798004e00900080
:106514000080fa00000006001400fa0060079800ea
:1065240071079800025798000000eb0030079800ac
:106534006e009000100f78006e00900070119000b3
:106544008019900012079800230798006e009000ad
:106554001e019000ae0190001218980023189800b4
:1065640012c0b300fe0090006e0090001bfb0700f9
:10657400500798005e0090000000e00003003a001d
:10658400c3012000130f98003e0037005e00900006
:1065940010407800004f98005e0090000000e0007a
:1065a400030032000e4890000004e00003003a00ab
:1065b400a000200030079800300037000e489000fb
:1065c400fb4f400003003a00a00020003007980071
:1065d4002a0037005e009000b0489000014f9800f8
:1065e400de00900050ceb300804878005e0090003a
:1065f4001d1f070010079800210798003e00900017
:106604000000e00005003a00fe0090006e009000db
:1066140019fa07000004e00003003a00100020000b
:106624003007980015003700c2788000d3788000c6
:106634001e009000ae009000820f5000838f58001f
:106644000e0032000e5090000004e0000b003200f7
:106654001e0178001e009000ae00900056fa07005c
:10666400804078000000eb00300798000104e0004f
:1066740002003a0010002000300798003e0190000c
:10668400120f98001e0890000080fa000000060017
:106694002600fa00881f7800700f980001179800f0
:1066a4000040eb00604f980010002000600f98003d
:1066b4000e1090000000e00092013a001083800068
:1066c4007011900080199000c0788000d17880000b
:1066d400800f5100818f590003003a000080eb00c5
:1066e400201798003c0237000040eb00704f9800e0
:1066f4000e0037007e4890000081fb007e48900029
:106704000080fb00800078007e089000008040003c
:106714009040780070004700000041000148780074
:106724007e4890000040e800704f98007e4890003a
:10673400ea4f500012003e007e4890000080fb00ab
:10674400800078007e0890000080400010407800af
:106754000004e000e7ff3a00090037007e4890009b
:106764008080fb00700047008080400000c2b300be
:10677400804878007e4890000040e800704f980000
:106784007e489000ea4f5000f4ff36007000470046
:106794008040eb00e7160700108380007011900022
:1067a40080199000320798004307980012838000f4
:1067b40010838000801890007010900010199800c9
:1067c4002119980010838000fc00470012c0b30018
:1067d40082fa070050079800188380005e0090003a
:1067e400a11e0700101c9800211c9800188380002b
:1067f4005e0090009c1e070070149800011c980015
:106804000000eb00600f980010838000fc0047003c
:1068140012c0b30071fa0700500798005e009000a0
:106824000000e00003003a008081eb002317980089
:10683400e90137000040eb00704f98001100370069
:106844007e4890008080fb005e0090000080400045
:10685400104178007e4890008080fb007000470063
:106864000080400010407800804f51000200320048
:1068740010c0b300604f98007e4890000040e800cc
:10688400704f98007e489000ea4f5000ecff3600ad
:106894006e4890000004e00003003a000080eb0022
:1068a40020179800cc0137000040eb00604f98009f
:1068b4005e0090006c1e0700107988002179880022
:1068c4003100370010838000fc0047000041eb00da
:1068d40042fa0700500798005e0090000000e000b4
:1068e40003003a008080eb0021179800ba013700ba
:1068f4000040eb00704f9800110037007e48900074
:106904008080fb005e009000008040001041780011
:106914007e4890008080fb007000470000804000ab
:1069240010407800804f51000200320010c0b300c4
:10693400604f98007e4890000040e800704f980037
:106944007e489000ea4f5000ecff36006e489000fd
:106954000004e00003003a000081eb0022179800d5
:106964009d0137000040eb00604f98006e089000d6
:106974000000e800600f98005e0090003a1e0700d7
:1069840010798800217988001279800023798000a9
:106994003e009000ce009000800f5100818f59007e
:1069a400c8ff3a0012798000237980003e009000ed
:1069b400ce009000800f5100818f59000c003a00e6
:1069c4005e00900010407800fb4f4000bdff320095
:1069d4005e00900030489000e84f5000b9ff32004c
:1069e4005e00900030489000ef4f5000b5ff320039
:1069f4006e0890000000e900600f98006e08900097
:106a0400600798000000e800600f98001083800081
:106a1400fc0047000041eb00f0f907005007980024
:106a24005e0090000000e00003003a008081eb006b
:106a340023179800680137005e009000104078002a
:106a44000004e000230032000040eb00704f980087
:106a5400110037007e4890008080fb005e009000ab
:106a640000804000104178007e4890008080fb0048
:106a7400700047000080400010407800804f5100b3
:106a84000200320010c0b300604f98007e489000ae
:106a94000040e800704f98007e489000ea4f500094
:106aa400ecff36006e4890000004e00003003a005a
:106ab4000080eb0020179800470137000040eb00ee
:106ac400604f98006e0890000000e800600f980086
:106ad400ceff3700ee009000610f98001283800013
:106ae4001083800080189000701090001019980096
:106af4002119980010838000fc00470012c0b300e5
:106b0400b6f90700500798000040eb00704f98005a
:106b140018003700128380007e4890008081fb00bb
:106b24007e4890008080fb00700047000080400099
:106b340090407800030041007c0040000148780048
:106b44007e4890000081fb007e4890008080fb001e
:106b54007000470000804000904078005e00900084
:106b640000004100014878007e4890000040e800a1
:106b7400704f98007e489000ea4f5000e5ff3600c1
:106b84001083800010199000a019900010838000d9
:106b9400100078005d030700100798002107980093
:106ba4006e0890004400de00004f780010838000df
:106bb40010007800405890000080fb0010179800e7
:106bc4001e119000e10f5100220035009e1190002b
:106bd400e28f51000e0034001e109000e30f5000ad
:106be400010032001b003700108380001000780081
:106bf400b05890001e80fb000181fb0011000900c9
:106c04000280d8008000fd00004f7800110037009a
:106c1400108380007011900080199000c07880006b
:106c2400d1788000800f5100818f59000900320013
:106c34001083800010007800b05890001e80fb0084
:106c44000181fb00110009000280d8008000fd00d2
:106c5400004f780010838000100078001002780044
:106c64001e4078000081fb00030020001e009000fd
:106c7400ae00900002004000838048008041eb0099
:106c840004017800e92807000004e00003003a004a
:106c94008080eb0021179800cf0037000040eb0004
:106ca400704f9800030037007e4890000040e800d1
:106cb400704f98007e4890008080fb007000470071
:106cc400008040009040780000c2b30080cf5000a4
:106cd400030032007e489000ea4f5000f2ff360075
:106ce4007e4890008080fb00700047008080400058
:106cf4000040eb0080487800700047004a0c070011
:106d0400b30037000e109000fc0040000041eb007f
:106d14007e0890009c0507000004e00003003a0090
:106d24000081eb0022179800ab0037000040eb0015
:106d3400704f98000e0037007e4890000081fb00e1
:106d44007e4890000080fb008e1090007c00400084
:106d540001004000904078007000470000004100ae
:106d6400014878007e4890000040e800704f980089
:106d74007e489000ea4f5000efff36000e1090005e
:106d8400c0119000630798000000eb00600f9800aa
:106d94000e10900080189000701090000e1190005a
:106da4001019980021199800fc00470012c0b30084
:106db4000e10900009f90700500798005e0090003b
:106dc4000000e00003003a000080eb002017980068
:106dd400810037000040eb00704f9800110037002d
:106de4007e4890008080fb005e00900000804000a0
:106df400104178007e4890008080fb0070004700be
:106e04000080400010407800804f510002003200a2
:106e140010c0b300604f98007e4890000040e80026
:106e2400704f98007e489000ea4f5000ecff360007
:106e34006e4890000004e00003003a008080eb00fc
:106e440021179800640037000040eb00604f980061
:106e5400fc0047000041eb000e109000dff8070033
:106e6400500798005e0090000000e00003003a0024
:106e74000081eb0022179800570037005e00900055
:106e8400104078000004e000230032000040eb00d2
:106e9400704f9800110037007e4890008080fb00fe
:106ea4005e00900000804000104178007e48900011
:106eb4008080fb0070004700008040001040780094
:106ec400804f51000200320010c0b300604f9800a0
:106ed4007e4890000040e800704f98007e48900083
:106ee400ea4f5000ecff36006e4890000004e000ca
:106ef40003003a008081eb00231798003600370026
:106f04000040eb00604f98006e0890000000e8001d
:106f1400600f9800ceff37006e009000600f98005d
:106f24000e10900080189000701090000e119000c8
:106f34001019980021199800fc0047000e109000c9
:106f440032fd0700500798005e0090000000e0004a
:106f540003003a008080eb00211798001e003700e0
:106f64000040eb00704f98000e0037007e48900000
:106f74000081fb007e4890000080fb008e10900092
:106f84007c00400001004000904078005e009000ca
:106f940000004100014878007e4890000040e8006d
:106fa400704f98007e489000ea4f5000efff360083
:106fb400fc0047000e109000aff707000004e0004b
:106fc40003003a000081eb0022179800020037000a
:106fd4008001eb00231798002e1090004f047800d6
:106fe4000080fa00000006001200fa005007980022
:106ff40061079800742807000004e00003003200d1
:107004000000eb00000f9800120137000000eb00b5
:10701400300798000000eb002007980016003700a6
:10702400ae009000a0f020000080400010407800e6
:107034000004e0000d003200ae009000a0f020003b
:10704400808040000040eb0080487800ae00900053
:10705400600320000088b9008000780080e62000ea
:107064000080400030079800060037002e00900092
:107074000000e800200798002e009000e20f500066
:10708400e7ff34003e0090000000e00003003a00f7
:107094008000eb00010f9800ee0037003e009000e6
:1070a400fc0040000041eb005e009000b6040700c5
:1070b4000004e00008003a00ae009000a0f02000b8
:1070c4008080400010c0b300804878000000eb00ce
:1070d400000f9800df0037006e0090001040780029
:1070e40020479800be009000e0fc20008008780053
:1070f4003e0190006000b800100198002101980042
:107104003e0190006000b8003001980041019800f1
:10711400be0090000000eb00c0109800be0090007c
:1071240000022000e0109800108380008018900076
:10713400701090003e0190007011980001199800a1
:1071440010838000a0189000101890003e01900059
:107154001019980021199800be00900020f6200014
:10716400300107008041eb0012c0b30021f620007b
:107174003e00900063f007000000e0007f003a004a
:107184002e4090000080fb007007980070052000de
:10719400fe009000808f50001a003200700520001d
:1071a400fe009000808f500009003c001004200075
:1071b400fe009000808f5000300032002005200037
:1071c400fe009000808f500060003200680037009d
:1071d40020072000fe009000808f50005b003200ea
:1071e40070072000fe009000808f500005003200e0
:1071f40010062000fe009000808f50001f00320017
:107204005b0037003e00900040109000400798005b
:10721400e800470012c0b3003e009000befc070027
:10722400000f78001e00e0007f003a00e8004700ed
:107234000041eb003e009000cdf80700000f7800fd
:107244001e00e00078003a00e800470072c7b3006f
:107254003e0090001af10700000f78001e00e000c5
:1072640071003a00210020006011b8003e00900037
:10727400db050700000f78006b0037003e0090002c
:10728400a008900010089000e00f5000e08f580014
:10729400100032003e00900040109000400798001b
:1072a400e800470072c7b3003e00900004f10700f5
:1072b400000f78001e00e0005b003a00210020006f
:1072c4006011b8003e009000c5050700000f78006b
:1072d400550037003e009000401090004007980091
:1072e400e800470012c0b3003e0090008afc07008b
:1072f400000f78001e00e0004b003a00e800470051
:107304000041eb003e00900099f80700000f780060
:107314001e00e00044003a00e800470072c7b300d2
:107324003e009000e6f00700000f78001e00e00029
:107334003d003a00210020006011b8003e0090009a
:10734400a7050700000f7800370037003e009000c3
:107354004010900040079800e800470022c7b3009f
:107364003e009000d6f00700000f78002e00370092
:10737400f00f2000000f78002b00370021f62000ca
:107384003e009000a7000700ae40900070c7b30015
:1073940080cf50000c003200ae40900070c5b300a6
:1073a40080cf500008003200ae40900010c6b300f9
:1073b40080cf500004003200ae40900010c4b300ef
:1073c40080cf500016003a000000eb004007980000
:1073d400e80047000041eb003e00900064f807001d
:1073e400000f78001e00e0000f003a00e80047009c
:1073f40072c7b3003e009000b1f00700000f7800a0
:107404001e00e00008003a00210020006011b800ce
:107414003e00900072050700000f7800020037005c
:10742400a0002000000f78001e00e00007003200da
:10743400ae009000a0f020008080400010c0b30097
:10744400804878000000eb00300798003e00900070
:10745400000f98000e0890000080fa00000006005b
:107464000200fa00000f78001e00780080089000e7
:10747400700090000080fa00000006000800fa0086
:1074840020079800c0f22000100798004e2707003c
:107494000004e000030032000080eb003007980095
:1074a400430037001e009000fc0040000041eb0048
:1074b4002e009000b40307000004e00003003a002b
:1074c4000080eb0030079800390037009e009000e0
:1074d400e0fc2000800878001e0190006000b800e5
:1074e40010019800210198001e0190006000b8006e
:1074f40030019800410198009e0090000000eb00cc
:10750400c01098009e00900000022000e010980037
:107514001083800080189000701090001e0190006d
:10752400701198000119980010838000a018900031
:10753400101890001e01900010199800211998004d
:107544009e00900020f62000360007008041eb00ea
:1075540012c0b30021f620001e00900069ef07005e
:10756400000f78001e00e000030032000080eb00f2
:10757400300798000e0037001e00900081022000a2
:107584008080400012c0b3001e009000e2fb0700a0
:10759400000f78001e00e00003003a000000eb003a
:1075a40030079800020037000080eb003007980095
:1075b4003e0090000080fa00000006000200fa007d
:1075c400000f78005ed0bf000004e000010032002c
:1075d4005b0207001e0178006000b800700198008b
:1075e400010998009e0078000000eb00e00098007c
:1075f4009e0078000000eb00d00098001e00780088
:10760400a0009000100090001e0178003001980046
:10761400410198000000eb00c08288000080fa005d
:10762400000006000a00fa0030079800410798009d
:107634003e009000100798004e009000000f780064
:1076440060c3b300404798000040eb0026efb7004a
:107654000d00370026cfbf000080fb0080007800bb
:107664001e0090008080400026cfbf000080fb00f9
:107674001e004000104078008048780026cfbf00ec
:107684000040e80026efb70061f220009140780046
:107694004e40900080cf5000eeff39000080fa0089
:1076a400000006000800fa0020079800310798003f
:1076b4000000eb00000f78002e009000900078008e
:1076c400110798002e0090005bf907003e0190001e
:1076d4000089be003e0090001000be00e00f500084
:1076e400e08f580003003a0020012000000f7800ca
:1076f4003f0037001e00900040589000e14f5000ba
:1077040010003a003e0090001001be008040eb00e3
:1077140084ff2000050020001e009000940707004d
:107724000001be00f0ff2f0001002000800f510077
:10773400818f590026003a0080002000000f780055
:10774400230037001e00900040589000e24f500084
:1077540010003a003e0090001001be008040eb0093
:1077640084ff2f00050020001e0090008007070002
:107774000001be00f0ff2f0001002000800f510027
:10778400818f590012003a0080002000000f780019
:107794000f0037003e0090001001be008040eb0057
:1077a40084ff2f00f5ff20001e00900070070700e3
:1077b4000001be00f0ff2f00f1ff2000800f5100f8
:1077c400818f590002003a0080002000000f7800e9
:1077d4001e00e00006003a003e0090001001be00ca
:1077e4001e009000050007000080fb00000f7800d9
:1077f4001e0078000080fa00000006001000fa0065
:107804004007980052079800630798000040eb0077
:10781400004f78005e019000ee0190004e00900051
:107824003a00070010079800210798005ed0bf00b7
:107834000004e00006003200c10107000004e0007b
:1078440003003200f00f2000700798002c0037006e
:107854000000eb00c08288005fd0bf000004e0009d
:1078640007003a004e00900010007800022020002b
:107874008000eb003dec070010c0b3005ff0b700e0
:107884000040eb0060479800140037004e00900061
:10789400100178001e029000ae0290001e009000bd
:1078a400ae00900061004000e0804800100798009e
:1078b400210798008041eb000400be00db2507008f
:1078c400e14f50000200320080c0b300004f780046
:1078d4006e4090000040e800604798004e00900021
:1078e400b05890006e40900080cf500002003600e7
:1078f4001e04e000e5ff32001e80fb0070079800c4
:107904007e0090000080fa00000006000c00fa00df
:10791400889fbe002007980032079800430798000c
:107924002e009000405890000080fb005007980003
:107934005e009000e10f5000440035005e009000ae
:10794400e20f5000190034005e009000e30f500075
:10795400010032003d0037003e009000ce00900050
:1079640062045000e08458002e00900030589000cb
:107974000081fb00030020000243b80003c0b900eb
:1079840007027800000242000990b9000002420098
:10799400840378002e00900080089000700090000e
:1079a400001f430001974b00280037003e00900061
:1079b400ce009000e00f5000e08f58000700320026
:1079c4003e019000ce019000100020000100200034
:1079d400800f5100818f590008003a002e0090005a
:1079e40050019000e00190003e009000ce00900015
:1079f400001f410001974900140037003e00900029
:107a0400ce00900062045000e08458002e009000e4
:107a1400305890000081fb00030020000243b800ae
:107a240003c0b90007027800000242000990b900bf
:107a340000024200840378002e0090008008900029
:107a440070009000001f430001974b001e00be0011
:107a54004f04be000080fa00000006002600fa0071
:107a6400600f9800710f9800021798001317980080
:107a7400fe0890000e1090000088b900010020005c
:107a8400400f9800510f98006e089000300f980036
:107a94000000eb00100f98000000eb0010079800a6
:107aa4001e10900030089000610060000000e000ab
:107ab40005003a0080002000100f98008000eb00c1
:107ac400211798001b0137004e089000de08900033
:107ad400e00f5000e08f580003003a000001eb0073
:107ae4002217980013013700b72507000004e000af
:107af4000500320060012000100f98008001eb00a7
:107b0400231798000b0137000040eb005ff0b7002b
:107b14001e10900090007800210f98001e10900015
:107b240060019000020f98001e10900070019000f8
:107b34008009900042079800530798001e10900097
:107b440030019000c00190002e0890006fff0700e4
:107b540060079800710798001e1090005000900074
:107b64006101b8006e009000fe009000000041002a
:107b7400818049006007980071079800c1828000e5
:107b84001e109000808f50000b0032005ed0bf00aa
:107b94000004e00006003200e90007000004e000f1
:107ba400030032008001eb0023179800e100370046
:107bb4001e109000c0828800d2828000e382800080
:107bc4006e009000fe009000800f5100818f5900dc
:107bd400180032005ed0bf000004e000060032004e
:107be400d70007000004e000030032008000eb002f
:107bf40021179800cf0037000040eb005ff0b7007a
:107c04002e089000100178006e009000fe00900095
:107c1400172407000004e00002003a00700020006e
:107c2400100f98006e019000fe019000d28288002f
:107c3400e38288001e10900010099000a0099000b3
:107c44002207980033079800a00037004e019000e7
:107c5400de0190002e009000be009000800f5100c5
:107c6400818f590004003a009e1090003108900062
:107c74000010a000b00898008e089000002020009a
:107c8400808f500065003a0010c0b300004f7800a8
:107c94005ed0bf000004e00006003200a800070028
:107ca4000004e000030032008081eb0023179800f9
:107cb400a00037000000eb00000f98001e10900099
:107cc400500090008000e8001e10900051009800c1
:107cd4001e109000d00090002e08900030589000a4
:107ce4000080fb00808f500016003a009e10900028
:107cf4000000eb00d00098001e10900030089000a7
:107d0400620060000000e000080032008040eb00e8
:107d14001e10900074f707000080fb00100f9800fd
:107d24000040eb00004f78000600370012002000ee
:107d3400030020001e109000f3ee07000080fb00fb
:107d4400100f98001e089000f20f500003003a0034
:107d54000000eb0020179800760037001e08900002
:107d64000000e0002d003a001e1090003001900049
:107d7400c00190002e089000e4fe07006007980000
:107d8400710798001e109000500090006101b80027
:107d94006e009000fe0090000000410081804900c8
:107da40060079800710798009e109000c1828800b7
:107db4001e04e000150032002e0890001001780027
:107dc4006e009000fe009000a92307000004e0006c
:107dd40009003a0070002000100f98000080eb00aa
:107de4008080eb00d0828800e18288000001eb00f3
:107df400221798004f0037006e009000fe0090009c
:107e0400d0828800e1828800040037006e0190006f
:107e1400fe019000d2828800e38288001e08900050
:107e24000000e00029003a002e089000900078003d
:107e34000e089000808040003e08900010407800ba
:107e4400804878000e0890000000e800000f9800b9
:107e54003e0890000000e800300f98004e009000ab
:107e6400de00900061004000e08048004007980078
:107e7400510798004e089000de0890006100500001
:107e8400e0805800400f9800510f98001e009000a9
:107e94000000e800100798001e10900030089000c1
:107ea400620060000000e000060032002e00900036
:107eb400be00900061004000e08048002007980068
:107ec4003107980010c0b3005ef0b7001e089000a0
:107ed4000000e00005003a004e089000de08900023
:107ee400e00f5000e08f580058ff3a001e10900039
:107ef4008e099000630098001e1090004e019000bf
:107f0400de01900072009800030898001e10900093
:107f14002e019000be0190001208980023089800da
:107f24001e0090007e099000110009000280d80014
:107f3400201798002e1090000080fa000000060020
:107f44000c00fa000000eb0010079800c0828000cb
:107f5400000f78001e007800900078002107980038
:107f64001e00780030019000c00190002e009000a7
:107f740066fe070030079800410798001e0078004d
:107f8400500090006101b8003e009000ce009000c7
:107f940000004100818049003007980041079800a3
:107fa4002e009000100178008041eb003e0090000c
:107fb400ce0090001d2407000004e00005003a00f4
:107fc4008000200010079800f00f20005007980050
:107fd400040037000040eb005ef0b7008000eb00c7
:107fe400510798005e0090000080fa00000006002f
:107ff4000400fa00000f78001e0078007001900061
:10800400800990001e007800a008900010089000dd
:108014000002eb0014079800800f5100818f590073
:1080240002003a0010002000100798001e00900083
:108034000080fa00000006002000fa00300f9800cb
:10804400410f9800520f9800630f9800ce089000db
:108054005e0890000088b90001002000100f98000d
:10806400210f98003e089000000f98000000eb00dc
:10807400100798000000eb00000f78006e089000d5
:1080840090007800710798006e08900060019000dd
:10809400220798006e0890007001900080099000fb
:1080a40052079800630798006e089000300890000b
:1080b400610060000000e000030032008001eb007a
:1080c400730f9800ad0037005ed0bf000004e000dd
:1080d400060032009aff07000004e00003003200ab
:1080e4000080eb00700f9800a4003700c18280006c
:1080f4006e089000808f50008e003200ae00900019
:1081040000202000808f50008a003200ee0890008a
:10811400c18288006e08900030019000c001900078
:108124007e009000f9fd0700300798004107980091
:108134006e089000500090006101b8003e0090006d
:10814400ce00900000004100818049003007980073
:10815400410798000040eb005ff0b7007e009000fc
:10816400100178003e009000ce009000c02207006d
:108174000004e00005003a00700020001007980099
:108184000001eb00720f98007c0037003e00900065
:10819400ce009000d0828800e1828800650037001c
:1081a4006e08900010099000a00990005e009000f5
:1081b400ee009000800f5100818f590003003a00b7
:1081c400d0032000100798005f003700ae00900035
:1081d40000202000808f50003c003a000000eb009b
:1081e400200798006e089000500090008000e8007e
:1081f4006e089000510098006e089000d000900026
:108204007e009000305890000080fb00808f50006a
:108214000c003a00ee0890000000eb00d00098003b
:1082240012002000030020006e089000b6ed070045
:108234000080fb00100798001e0090000000e00082
:1082440041003a006e08900030019000c001900097
:108254007e009000adfd07003007980041079800ac
:108264006e089000500090006101b8003e0090003c
:10827400ce00900000004100818049003007980042
:1082840041079800ee089000c18288000040eb008e
:108294005ff0b7007e009000100178003e0090006f
:1082a400ce009000722207000004e00003003a00b0
:1082b4007000200010079800230037003e01900052
:1082c400ce019000d2828800e38288007e00900074
:1082d400900078002e0090000080400090407800cc
:1082e4000e089000014878002e0090000000e8007d
:1082f400200798000e0890000000e800000f980086
:108304005e009000ee00900061004000e0804800b4
:1083140050079800610798001e0fe8001e0890009f
:10832400ae08900061005000e0805800100f9800e3
:10833400210f98001e089000ae089000e00f500036
:10834400e08f580096ff3a006e089000ae0190004e
:10835400630098006e0890005e019000ee019000aa
:1083640072009800030898001e0078004e099000df
:10837400110009000280d800700f98007e08900058
:108384000080fa00000006001e00fa00881f780032
:10839400300f9800410f9800225f98000040eb00d6
:1083a400004f7800070037001e80fb008000780033
:1083b4004e0890008080400000c2b30080487800de
:1083c4001e4fe800a0c0b3009e4f1000f6ff360019
:1083d4003e08900090407800e0c2b30080cf500087
:1083e400040032003e089000104078000004e000d1
:1083f40003003a000000eb00600f980061003700b2
:108404003e0890007ae90700100798001e009000cb
:10841400ec0f50000a003e0066004700be089000c2
:108424007ae90700660047002e5990008040eb006f
:10843400580007000004e000040032000600370082
:108444000000eb00600f98004e0037000000eb00c6
:10845400600f98004b00370066004700e1022000df
:1084640072e90700200798002e0090000000e00049
:108474000d003200ae0090000040eb008048780010
:108484002e0090000000e800200798002e009000c5
:1084940057e90700e30f5000030036000000eb002b
:1084a400600f9800370037006600470050e9070066
:1084b400e80f5000030036000000eb00600f980046
:1084c400300037000040eb00004f78000b0037000d
:1084d4001e80fb00800078004e0890000081400060
:1084e4001e80fb0080007800660047000100400009
:1084f40010407800004978001e4fe8001e84fb00fd
:10850400660047003ae90700800f5400f0ff390085
:108514002e0090000000e000180032002e009000b1
:10852400104078000004e000140032000040eb002a
:10853400004f78000c0037001e80fb00800078009c
:108544004e08900000804000680140001e80fb003f
:10855400800078002e0090000080400010407800d9
:10856400004978001e4fe8001e84fb002e00900096
:108574001fe90700800f5400efff390010002000ae
:10858400600f98006e0890004f0478000080fa0095
:10859400000006000e00fa00881f780020079800eb
:1085a40061479800724798002e00900010e9070078
:1085b400100798000000eb00000f78004d00370012
:1085c4006e4090000004e00023003a001e00780092
:1085d400800078002e009000008040001040780059
:1085e400fe4090004c0007000080fb0060079800ec
:1085f4006e009000e10f5000070032006e00900002
:10860400e10f50003a0035006e009000e30f500077
:1086140037003c000d0037001e0078008000780011
:108624002e009000008440001e0078008000780036
:108634002e00900000804000104078000000fb00f5
:10864400e4e80700004c7800290037000000eb0044
:10865400500798002c0037006e409000e14f500006
:1086640023003a001e007800800078002e0090005d
:108674000080400010407800fe4090008200070017
:108684000080fb00400798004e0090000000e000ce
:10869400040032004e009000e10f50000800320048
:1086a400130037001e007800800078002e00900030
:1086b40080804000f0c5b300804878000c0037008b
:1086c4001e007800800078002e0090000084400096
:1086d4001e007800800078002e009000008040008a
:1086e400104078000000fb00bae80700004c780056
:1086f4001e0fe8001e0090009e0f1000b0ff350012
:1087040010002000500798005e0090004f0478008d
:108714000080fa00000006000400fa00004f780010
:108724001147980000c4b3009e4f100003003400aa
:10873400a0c5b3009e4f100033003400f0c2b30054
:108744009e4f10000300340090c3b3009e4f1000ee
:108754002d00340040c2b3009e4f10002a003200a6
:1087640050c2b3009e4f10002700320070c2b30005
:108774009e4f100024003200d0c2b3009e4f100060
:1087840021003200f0c5b3009e4f10001e003200dd
:1087940000c4b3009e4f10001b003200e0c7b300ba
:1087a4009e4f10001800320000c6b3009e4f100008
:1087b4001500320010c2b3009e4f100012003200a8
:1087c40080c2b3009e4f10000f00320090c2b3006d
:1087d4009e4f10000c003200e0c5b3009e4f100005
:1087e4000900320030c2b3009e4f10000600320070
:1087f40060c2b3009e4f100003003200e0c2b30019
:108804009e4f100003003a000000eb001007980090
:108814001a00370000c6b3009e4f10000600340053
:10882400a0c7b3009e4f100003003c0010002000be
:1088340010079800110037001e4090000004e0006b
:1088440006003200a0c2b3009e4f100003003a009d
:108854000000eb00100798000800370000c2b300c6
:108864009e4f100003003a003000200010079800cb
:108874000200370020002000100798001e0090001e
:108884000080fa00000006000400fa00004f78009f
:10889400114798001e4090000004e00006003200da
:1088a400a0c2b3009e4f100003003a002000200035
:1088b4001007980047003700f0c1b3009e4f100026
:1088c40003003e0050c0b3009e4f100033003a0036
:1088d40020c2b3009e4f100030003200a0c2b3008b
:1088e4009e4f10002d003200b0c2b3009e4f100006
:1088f4002a003200c0c2b3009e4f1000270032008d
:10890400e0c2b3009e4f100024003200f0c2b30056
:108914009e4f100021003200a0c3b3009e4f1000f0
:108924001e003200b0c3b3009e4f10001b00320083
:10893400c0c3b3009e4f100018003200d0c3b30070
:108944009e4f100015003200e0c3b3009e4f10008c
:1089540012003200f0c3b3009e4f10000f0032002b
:10896400b0c5b3009e4f10000c003200c0c5b30068
:108974009e4f100009003200d0c5b3009e4f100076
:1089840006003200c0c7b3009e4f1000030032003f
:108994001e4078000004e00003003d000000eb00ee
:1089a400100798000b00370000c6b3009e4f10005c
:1089b40006003600a0c7b3009e4f100003003e001f
:1089c400100020001007980002003700200020004b
:1089d400100798001e0090000080fa0000000600b6
:1089e4001c00fa006007980072079800030f9800b3
:1089f400110f98006e009000900078001107980005
:108a04001e099000320f9800be099000e18f5100ba
:108a1400040032003e0a9000e20f52000b003200c4
:108a2400130037006e0090007001900080099000e0
:108a34007e0090008e089000020040008380480071
:108a440070079800010f9800090037006e0090002d
:108a540010099000a00990007e0090008e089000fc
:108a6400000051008180590070079800010f9800a0
:108a74005ed0bf000004e0000600320030fd0700b5
:108a84000004e000030032000080eb00200f980097
:108a9400e00037006e00900010019000a0019000eb
:108aa40022079800330798006e0090002e01900072
:108ab400be01900032009800430098006e009000c0
:108ac40010099000a009900022079800330798002d
:108ad4007e0190008e0990002e009000be00900050
:108ae400800f5100818f5900030036008081eb0014
:108af400230f9800c7003700ee0090003108900063
:108b04000010a100b00898007e0090008e0890002c
:108b14006e01900070019800010998007e00900099
:108b24008e089000400f9800510f98004e08900056
:108b3400de089000e00f5000e08f580006003d0072
:108b44004e099000de099000f21fb0000380b000cf
:108b5400420f9800530f98004e099000de099000d0
:108b6400471add004910de0000007200c998de00db
:108b740040079800510798007e0190008e099000ec
:108b84004e009000de009000490add00c700de00c0
:108b9400810072004900dd0000005100818059000d
:108ba40070079800010f9800fe0090006e0090007e
:108bb400610098001e009000305890000081fb0076
:108bc400030020004e009000de009000a0e70700a4
:108bd40020079800310798001e009000305890003c
:108be4000082fb00050020002e0090000023b80046
:108bf4003e00900000a0b900070178000001410088
:108c04002e0090000580b900000141008203780025
:108c14004e009000de00900006005000878058004f
:108c24004007980051079800ce0090006e00900015
:108c3400510098002e009000be009000e00f5000fc
:108c4400e08f58004b0032002e019000be019000ce
:108c54006e0090002ceb0700004f78001e04e0002b
:108c640044003200c0c3b3009e4f10003e003a00df
:108c74006e00900030089000610060000000e00089
:108c84001c0032006e009000a000900010009000c4
:108c94006e01900030019800410198002e0190006f
:108ca400be0190001000200001002000800f510040
:108cb400818f5900070032002e009000be00900002
:108cc40061015000e08158006e0090000eeb070037
:108cd400004f78008040eb006e00900082f30700a4
:108ce4000004e000230032000080eb00200f980015
:108cf400480037006e009000a00090001000900023
:108d04006e01900030019800410198002e009000ff
:108d1400be00900061015000e08158006e00900098
:108d2400f9ea0700004f78001e04e0000300320057
:108d34008080eb00210f980036003700ee00900091
:108d440000202000e00098001e00900030589000a1
:108d54000080fb000000e900800078006e009000b5
:108d640051009800030037000081eb00220f9800a7
:108d7400280037006e00900030019000c001900080
:108d84001e009000e1fa07002007980031079800c0
:108d94006e009000500090000100200040079800f1
